:06000000020033020E664F
:03000B00020E677B
:03001300020E8159
:03001B00020E8250
:03002300020E8347
:03002B00020E843E
:10003300759840758780758921758DFF758BFF7560
:100043008850D299758160758CFA758A0075A8827B
:1000530075900075B0FF7535FF7537FF7539FF75FE
:100063003BFF753DFF753FFF7541FF7543FF7545C9
:10007300FF753600753800753A00753C00753E0013
:1000830075400075420075440075300C753100D21F
:10009300A0D2A1782076FF08B830FAC2A27E80DF12
:1000A300FEDEFCC280C287C286D285D284D2A3C2BE
:1000B300A3DFFEDFFEDFFEDFFEDFFED2A3C2A3DF90
:1000C300FED2A3C2A3DFFEC284D2A3C2A3742812AA
:1000D300108FDFFE740812108FDFFE740612108F6C
:1000E300DFFE741012108FDFFE740C12108FDFFE10
:1000F300740112108FDFFEDFFE744012108F7F40F9
:10010300901328E4931210B4A3DFF8748012108FB5
:100113007F14901368E4931210B4A3DFF874C01231
:10012300108F7F1490137CE4931210B4A3DFF8DFD5
:10013300FEDEFCDFFEDEFCDFFEDEFCDFFEDEFC744B
:100143008012108F7F14901390E4931210B4A3DFE6
:10015300F874C012108F7F149013A4E4931210B498
:10016300A3DFF8759000D2A0D2A17880E670257540
:10017300B0FE75A00120A00F300019C200760890D0
:10018300119C120F25800D20000AD20076089011D1
:100193009F120F257881E6702575B0FE75A00220A9
:1001A300A10F300119C20176089011A2120F258008
:1001B3000D20010AD20176089011A5120F2578901F
:1001C300E6702575B0FB75A00120A00F301019C291
:1001D3001076089011A8120F25800D20100AD21056
:1001E30076089011AB120F257891E6702575B0FB58
:1001F30075A00220A10F301119C21176089011AE1B
:10020300120F25800D20110AD21176089011B11218
:100213000F257898E6702575B0F775A00120A00F1B
:10022300301819C21876089011B4120F25800D20CA
:10023300180AD21876089011B7120F257899E6702C
:100243002575B0F775A00220A10F301919C21976D0
:10025300089011BA120F45800D20190AD219760899
:100263009011BD120F4578A0E6702575B0EF75A00B
:100273000120A00F302019C22076089011C0120F60
:1002830025800D20200AD22076089011C3120F2555
:1002930075B0EF75A00220A126753207120E9312D6
:1002A3000E85D53206753201120E93120E8C75B07F
:1002B300EF75A00220A10820190302116580E378DD
:1002C300A8E6702575B0DF75A00120A00F302819AE
:1002D300C22876089011C6120F25800D20280AD255
:1002E3002876089011C9120F2575B0DF75A002207A
:1002F300A126753207120EB8120E85D53206753255
:1003030001120EB8120E8C75B0DF75A00220A10881
:1003130020190302116580E378B0E6702575B0BF3C
:1003230075A00120A00F303019C23076089011CC8F
:10033300120F25800D20300AD23076089011CF128B
:100343000F2575B0BF75A00220A120753207120ECC
:10035300DD120E85D53206753201120EDD120E8CBA
:1003630075B0BF75A00220A10280E978B8E67025B8
:1003730075B07F75A00120A00F303819C2387608F8
:100383009011D2120F25800D20380AD238760890AA
:1003930011D5120F2575B07F75A00220A1207532EB
:1003A30007120F01120E85D53206753201120F01A5
:1003B300120E8C75B07F75A00220A10280E97590A2
:1003C300FFC2A0C2A178C0E6702575B0FE7590018A
:1003D30020900F304019C24076089011D8120F2593
:1003E300800D20400AD24076089011DB120F257849
:1003F300C1E6702575B0FE75900220910F3041194A
:10040300C24176089011DE120F25800D20410AD2D9
:100413004176089011E1120F2578C2E6702575B078
:10042300FE75900420920F304219C2427608901153
:10043300E4120F25800D20420AD24276089011E77C
:10044300120F2578C3E6702575B0FE7590082093CA
:100453000F304319C24376089011EA120F25800D1D
:1004630020430AD24376089011ED120F2578C4E693
:10047300702575B0FE75901020940F304419C24456
:1004830076089011F0120F25800D20440AD244768D
:10049300089011F3120F2578C5E6702575B0FE7527
:1004A300902020950F304519C24576089011F61219
:1004B3000F25800D20450AD24576089011F9120FB9
:1004C3002578C6E6702575B0FE75904020960F30EE
:1004D3004619C24676089011FC120F25800D20465E
:1004E3000AD24676089011FF120F2578C7E67025C9
:1004F30075B0FE75908020970F304719C247760874
:10050300901202120F25800D20470AD247760890D9
:100513001205120F2578D0E6702575B0FB75900192
:1005230020900F305019C2507608901208120F25F0
:10053300800D20500AD250760890120B120F2578A6
:10054300D1E6702575B0FB75900220910F305119DB
:10055300C251760890120E120F25800D20510AD237
:10056300517608901211120F2578D2E6702575B0D6
:10057300FB75900420920F305219C25276089012E4
:1005830014120F25800D20520AD2527608901217AA
:10059300120F2578D3E6702575B0FB75900820936C
:1005A3000F305319C253760890121A120F25800D7B
:1005B30020530AD253760890121D120F2578D4E6E1
:1005C300702575B0FB75901020940F305419C254E8
:1005D3007608901220120F25800D20540AD25476EB
:1005E30008901223120F2578D5E6702575B0FB7598
:1005F300902020950F305519C25576089012261277
:100603000F25800D20550AD2557608901229120F16
:100613002578D6E6702575B0FB75904020960F308F
:100623005619C256760890122C120F25800D2056AB
:100633000AD256760890122F120F2578D7E6702526
:1006430075B0FB75908020970F305719C257760805
:10065300901232120F25800D20570AD25776089038
:100663001235120F2578D8E6702575B0F77590010D
:1006730020900F305819C2587608901238120F255F
:10068300800D20580AD258760890123B120F257815
:10069300D9E6702575B0F775900220910F3059197E
:1006A300C259760890123E120F25800D20590AD2A6
:1006B300597608901241120F2578DAE6702575B045
:1006C300F775900420920F305A19C25A7608901287
:1006D30044120F25800D205A0AD25A7608901247E9
:1006E300120F2578DBE6702575B0F7759008209317
:1006F3000F305B19C25B760890124A120F25800DEA
:10070300205B0AD25B760890124D120F2578DCE647
:10071300702575B0F775901020940F305C19C25C8A
:100723007608901250120F25800D205C0AD25C7659
:1007330008901253120F2578DDE6702575B0F77512
:10074300902020950F305D19C25D760890125612E5
:100753000F25800D205D0AD25D7608901259120F85
:100763002578DEE6702575B0F775904020960F303A
:100773005E19C25E760890125C120F25800D205E12
:100783000AD25E760890125F120F2578DFE6702595
:1007930075B0F775908020970F305F19C25F7608A8
:1007A300901262120F25800D205F0AD25F760890A7
:1007B3001265120F2578E0E6702575B0EF7590018C
:1007C30020900F306019C2607608901268120F25CE
:1007D300800D20600AD260760890126B120F257884
:1007E300E1E6702575B0EF75900220910F30611925
:1007F300C261760890126E120F25800D20610AD215
:10080300617608901271120F2578E2E6702575B0B3
:10081300EF75900420920F306219C262760890122D
:1008230074120F25800D20620AD262760890127727
:10083300120F2578E3E6702575B0EF7590082093C5
:100843000F306319C263760890127A120F25800D58
:1008530020630AD263760890127D120F2578E4E6AE
:10086300702575B0EF75901020940F306419C26431
:100873007608901280120F25800D20640AD26476C8
:1008830008901283120F2578E5E6702575B0EF7591
:10089300902020950F306519C26576089012861254
:1008A3000F25800D20650AD2657608901289120FF4
:1008B3002578E6E6702575B0EF75904020960F30E9
:1008C3006619C266760890128C120F25800D206679
:1008D3000AD266760890128F120F2578E7E6702504
:1008E30075B0EF75908020970F306719C26776084F
:1008F300901292120F25800D20670AD26776089016
:100903001295120F2578E8E6702575B0DF75900112
:1009130020900F306819C2687608901298120F253C
:10092300800D20680AD268760890129B120F2578F2
:10093300E9E6702575B0DF75900220910F306919D3
:10094300C269760890129E120F25800D20690AD283
:100953006976089012A1120F2578EAE6702575B022
:10096300DF75900420920F306A19C26A76089012DC
:10097300A4120F25800D206A0AD26A76089012A766
:10098300120F2578EBE6702575B0DF75900820937C
:100993000F306B19C26B76089012AA120F25800DC7
:1009A300206B0AD26B76089012AD120F2578ECE615
:1009B300702575B0DF75901020940F306C19C26CE0
:1009C30076089012B0120F25800D206C0AD26C7637
:1009D300089012B3120F2578EDE6702575B0DF7518
:1009E300902020950F306D19C26D76089012B612C3
:1009F3000F25800D206D0AD26D76089012B9120F63
:100A03002578EEE6702575B0DF75904020960F309F
:100A13006E19C26E76089012BC120F25800D206EDF
:100A23000AD26E76089012BF120F2578EFE6702572
:100A330075B0DF75908020970F306F19C26F7608FD
:100A43009012C2120F25800D206F0AD26F76089084
:100A530012C5120F2578F0E6702575B0BF759001A9
:100A630020900F307019C27076089012C8120F25AB
:100A7300800D20700AD27076089012CB120F257861
:100A8300F1E6702575B0BF75900220910F30711992
:100A9300C27176089012CE120F25800D20710AD2F2
:100AA3007176089012D1120F2578F2E6702575B091
:100AB300BF75900420920F307219C272760890129B
:100AC300D4120F25800D20720AD27276089012D7A5
:100AD300120F2578F3E6702575B0BF759008209343
:100AE3000F307319C27376089012DA120F25800D36
:100AF30020730AD27376089012DD120F2578F4E67C
:100B0300702575B0BF75901020940F307419C2749E
:100B130076089012E0120F25800D20740AD27476A5
:100B2300089012E3120F2578F5E6702575B0BF75AE
:100B3300902020950F307519C27576089012E61231
:100B43000F25800D20750AD27576089012E9120FD1
:100B53002578F6E6702575B0BF75904020960F3066
:100B63007619C27676089012EC120F25800D207646
:100B73000AD27676089012EF120F2578F7E67025E1
:100B830075B0BF75908020970F307719C2777608BC
:100B93009012F2120F25800D20770AD277760890F3
:100BA30012F5120F2578F8E6702575B07F75900160
:100BB30020900F307819C27876089012F8120F251A
:100BC300800D20780AD27876089012FB120F2578D0
:100BD300F9E6702575B07F75900220910F30791971
:100BE300C27976089012FE120F25800D20790AD261
:100BF300797608901301120F2578FAE6702575B0FF
:100C03007F75900420920F307A19C27A7608901378
:100C130004120F25800D207A0AD27A7608901307E2
:100C2300120F2578FBE6702575B07F759008209329
:100C33000F307B19C27B760890130A120F25800DA3
:100C4300207B0AD27B760890130D120F2578FCE6E1
:100C5300702575B07F75901020940F307C19C27C7D
:100C63007608901310120F25800D207C0AD27C7613
:100C730008901313120F2578FDE6702575B07F7564
:100C8300902020950F307D19C27D7608901316129F
:100C93000F25800D207D0AD27D7608901319120F3F
:100CA3002578FEE6702575B07F75904020960F304D
:100CB3007E19C27E760890131C120F25800D207EAC
:100CC3000AD27E760890131F120F2578FFE670254F
:100CD30075B07F75908020970F307F19C27F76089B
:100CE300901322120F25800D207F0AD27F76089061
:100CF3001325120F257590FFD2A0D2A17580FFD2C4
:100D0300A27407B535037535FF0535E535A2E092C5
:100D1300A4A2E192A5A2E292A6C2AFD2A7C2A7E47F
:100D2300B53503020D5604B53503020D7704B53509
:100D330003020D9804B53503020DB904B53503025A
:100D43000DDA04B53503020DFB04B53503020E1CA1
:100D5300020E3DE580F536A837A936120F6340062B
:100D630024FE500D8005120F685006853637120F8A
:100D73006F020E5EE580F538A839A938120F63407B
:100D83000624FE500D8005120F685006853839126F
:100D93000F93020E5EE580F53AA83BA93A120F6362
:100DA300400624FE500D8005120F685006853A3B1D
:100DB300120FB7020E5EE580F53CA83DA93C120F69
:100DC30063400624FE500D8005120F685006853CD3
:100DD3003D120FDB020E5EE580F53EA83FA93E12F1
:100DE3000F63400624FE500D8005120F68500685E0
:100DF3003E3F120FFF020E5EE580F540A841A94079
:100E0300120F63400624FE500D8005120F68500632
:100E1300854041121023020E5EE580F542A843A9E6
:100E230042120F63400624FE500D8005120F6850D6
:100E330006854243121047020E5EE580F544A8453D
:100E4300A944120F63400624FE500D8005120F685B
:100E5300500685444512106B020E5ED2AF02016646
:100E630002003332C0D0C0E0C0007880E6600116D3
:100E730008B800F8758CFAD000D0E0D0D032323206
:100E830032327E20DFFEDEFC227E60DFFEDEFC22CD
:100E9300748012108F05307419B53003753000E576
:100EA300307F049013B8E5302323931210B4A3DFEB
:100EB300F512118322748012108F153074FFB53030
:100EC30003753018E5307F049013B8E5302323937E
:100ED3001210B4A3DFF5121183223099FDC2997564
:100EE30099C074C012108F3099FDC2990531748076
:100EF300B53103753100E531F599121105223099A9
:100F0300FDC2997599C074C012108F3099FDC299B2
:100F1300153174FFB5310375317FE531F599121140
:100F23000522E4933099FDC299F599A3E493253002
:100F33003099FDC299F599A3E4933099FDC299F5CF
:100F43009922E4933099FDC299F599A3E4933099DA
:100F5300FDC299F599A3E4933099FDC299F59922BD
:100F6300C2D7E89922C2D7E99824FE223099FDC25C
:100F7300997599B074D112108F3099FDC2997599F2
:100F83005A3099FDC299E536C313F599121105221A
:100F93003099FDC2997599B0748D12108F3099FDF7
:100FA300C2997599553099FDC299E538C313F599DE
:100FB300121105223099FDC2997599B074891210E6
:100FC3008F3099FDC2997599533099FDC299E53ACD
:100FD300C313F599121105223099FDC2997599B081
:100FE300748512108F3099FDC2997599523099FD0D
:100FF300C299E53CC313F599121105223099FDC23C
:10100300997599B074C912108F3099FDC299759969
:10101300583099FDC299E53EC313F5991211052283
:101023003099FDC2997599B074C512108F3099FD2E
:10103300C2997599573099FDC299E540C313F59943
:10104300121105223099FDC2997599B0749112104D
:101053008F3099FDC2997599563099FDC299E54231
:10106300C313F599121105223099FDC2997599B0F0
:1010730074CD12108F3099FDC2997599593099FD2D
:10108300C299E544C313F59912110522C2A2C28085
:10109300339287339286339285339284D2A3C2A349
:1010A300339287339286339285339284D2A3C2A339
:1010B30022C2A2D2803392873392863392853392AF
:1010C30084D2A3C2A3339287339286339285339219
:1010D30084D2A3C2A32275F0648424301210B474A2
:1010E3000AC5F08424301210B4E5F024301210B491
:1010F3002275F00A8424301210B4C5F02430121083
:10110300B422D2D575F064847004C2D574F024304F
:101113001210B4740AC5F084700520D50274F0244B
:10112300301210B4E5F024301210B42275F00A84A2
:10113300700274F024301210B4E5F024301210B4AD
:1011430022E493A3B45E01221210B402114470048A
:101153007420800AC313C313C313C313C31312101E
:10116300B4221211833099FDC2997599B03099FD5B
:10117300C2997599783099FDC29975990002003327
:101183003099FDC2997599B03099FDC29975997BD3
:101193003099FDC29975990022905040805000907B
:1011A30051408051009052408052009053408053F0
:1011B30000905440805400B0407FB04000905540B0
:1011C30080550090564080560090574080570090BD
:1011D300584080580090184080180090194080199A
:1011E30000901A40801A00901B40801B00901C4006
:1011F300801C00901D40801D00901E40801E0090AA
:101203001F40801F009020408020009021408021BB
:1012130000902240802200902340802300902440AD
:101223008024009025408025009026408026009051
:10123300274080270090284080280090294080295B
:1012430000902A40802A00902B40802B00902C4055
:10125300802C00902D40802D00902E40802E0090F9
:101263002F40802F009030408030009031408031FB
:1012730000903240803200903340803300903440FD
:1012830080340090354080350090364080360090A1
:10129300374080370090384080380090394080399B
:1012A30000903A40803A00903B40803B00903C40A5
:1012B300803C00903D40803D00903E40803E009049
:1012C3003F40803F0090404080400090414080413B
:1012D300009042408042009043408043009044404D
:1012E30080440090454080450090464080460090F1
:1012F30047408047009048408048009049408049DB
:1013030000904A40804A00904B40804B00904C40F4
:10131300804C00904D40804D00904E40804E009098
:101323004F40804F00000000000000001F0000003D
:101333000000001F1F00000000001F1F1F0000000F
:10134300001F1F1F1F0000001F1F1F1F1F00001F64
:101353001F1F1F1F1F001F1F1F1F1F1F1F1F1F1FB9
:101363001F1F1F1F1F4D757A796B616E7420372005
:1013730076312E30612020202020736D69616C65E9
:101383006B2E7072762E706C20202020202043203C
:101393002020313237203132372031323720313279
:1013A300372020302020313237203132372031327C
:1013B30037203132372D4320202D4465732D4420AF
:1013C300202D4573202D4520202D4620202D4765B7
:1013D300732D4720202D4173202D4120202D4220A5
:1013E300202D482020204320202B4369732B4420A9
:1013F300202B4469732B4520202B4620202B466944
:10140300732B4720202B4769732B4120202B4169E5
:10141300732B4820202B432020204D757A796B6154
:101423006E7420372076312E306120323030372DE4
:1014330030372D3034202863294164616D20536D8A
:1014430069616C656B206A616E6B6F6D757A796B20
:10145300616E744077702E706C207777772E736D82
:1014630069616C656B2E7072762E706C2057737A7F
:10147300656C6B6965207072617761207A61737442
:10148300727A657A6F6E652E204A616B69656B6F40
:101493006C7769656B207A6173746F736F77616EB4
:1014A3006961206B6F6D657263796A6E65206B6F1E
:1014B3006475206E6965646F7A776F6C6F6E652EE5
:1014C30020416C6C205269676874732052657365A0
:1014D300727665642E204672656520666F72206E93
:1014E3006F6E20636F6D6D65726369616C206F6EE3
:0414F3006C792E20C2
:00000001FF
